:1000000000308A0052280000FF00030E8301A60082
:100010007F08A5000A08AD008A01A50E0408A70004
:100020002008A8002108A9002208AA002308AB0084
:100030002408AC00831383128C308400001C222817
:100040000C183528270884002808A0002908A100DA
:100050002A08A2002B08A3002C08A4002D088A005F
:10006000260E8300FF0E7F0E09008A113728AF0B82
:100070003C28AE0A0830AF000C108A112228463006
:1000800084000008031951280230A100A001A00B30
:100090004728A10B46289730A000A00B4D28800BC5
:1000A0004428003484011F3083051F130030831659
:1000B0009100073083129900713083168F000F086A
:1000C000831291110C3093002230960090309700EB
:1000D000AE010830AF00B001B101B201B301B4010B
:1000E000B501B601B701B801B901BA01BB01BC0144
:1000F000BD01BE01BF01C001C101C201C301C401F4
:10010000C501A53090008F018E0183160C14C030FC
:1001100083128B040730990083160508063083127A
:10012000A000A00B9128000019088C1183161F163F
:100130009F161F1383129F131F141F130030E738DD
:100140008316910000308312A1001F08C3392104D7
:100150009F008316851283128512B301B201320803
:10016000073C031C9629320DA000A00DFC30A00511
:100170001F08C33920049F000630A000A00BBE2832
:1001800000003630320784009F149F18C5281E08CF
:100190008000B208031D1F293E303207840080080A
:1001A000031D1F293630320784003008000203196E
:1001B0001F293630320784000008B0003008093C9F
:1001C000031CE5280130B1001F2930080A3C031C3C
:1001D000EB280030EC2801301D3C031CF2280230D3
:1001E000B1001F2930081F3C031CF8280030F928F3
:1001F0000130313C031CFF280330B1001F293008B7
:10020000333C031C0529003006290130453C031C02
:100210000C290430B1001F293008473C031C122967
:10022000003013290130593C031C19290530B10055
:100230001F2930085B3C03181F290630B1003630F7
:100240003207840000085E3C031C79293E303207E7
:1002500084008008031D7929B20803195429320843
:10026000023C031C5429B30803193F298316851245
:10027000831285120A30C6003F20AE01B3013E3022
:10028000320784000130800090308C1C4529950095
:100290000D303207C60046088C1C4C2995007F3073
:1002A0008C1C5029950078293208043C03187829C1
:1002B000B3080319642983168512831285120A3044
:1002C000C6003F20AE01B3013E303207840001304A
:1002D000800090308C1C6A2995000B303207C600D4
:1002E00046088C1C712995007F308C1C752995005F
:1002F0008A2936303207840000089F3C03188A2977
:100300003E3032078400800803198A293E303207C4
:10031000840080012E083B3C031894298316851223
:10032000831285160130B300B20AAF28AE286300ED
:02400E00C43FAD
:00000001FF
